:1000000001289401950183168B131F308500013060
:10001000860083128501860101309100E0200615DB
:10002000861701309100E020861306110611013079
:10003000003C0319D7288613FE2094008617203031
:1000400095000508113C0130031D0301003C031914
:100050002B28313095000508123C0130031D0301A7
:10006000003C03193528323095000508133C013057
:10007000031D0301003C03193F2833309500050898
:10008000143C0130031D0301003C0319492834309E
:1000900095000508153C0130031D0301003C0319C0
:1000A0005328353095000508163C0130031D030127
:1000B000003C03195D28363095000508173C0130D7
:1000C000031D0301003C031967283730950005081C
:1000D000183C0130031D0301003C0319712838301E
:1000E00095000508193C0130031D0301003C03196C
:1000F0007B283930950005081A3C0130031D0301A7
:10010000003C031985283030950005081B3C013060
:10011000031D0301003C03198F282A3095000508B0
:100120001C3C0130031D0301003C031999282330B6
:10013000950005081D3C0130031D0301003C031917
:10014000A3284130950005081E3C0130031D030122
:10015000003C0319AD28423095001408543C01308E
:10016000031D0301003C0319B82806154B301A2162
:100170001408523C0130031D0301003C0319C3283D
:1001800006114B301A211408433C0130031D0301B2
:10019000003C0319CD2815081A211408493C0130E8
:1001A000031D0301003C0319D628D7201728061584
:1001B000861701309100E0206521861306110800A2
:1001C000FA308D00EF20FA308D00EF20FA308D00EC
:1001D000EF20FA308D00EF20910BE02808008E30E0
:1001E0008E000000000000000000000000008E0BE8
:1001F000F32800008D0BEF2800000800083096005F
:100200009701061C01291021061C01291521970CB4
:10021000971706189713960B06291521170808003B
:1002200043309300930B1229080086309300930B00
:100230001729080099000930980086140000000072
:100240001521980B2629861015210800990C031CEE
:100250002B2986102029861420291008003C013003
:10026000031C3A290030031D3A290F08013C0130D4
:1002700003180301003C03194D2910088C000F08D6
:100280008F030F0A031990031A0892004E210617D4
:100290001A0892004E2106132D290800920C920C88
:1002A0003F309205033092020000920B5429000067
:1002B0000800FF309A008C01F0308F000C0890008D
:1002C0002D2146308D00EF200800FF308D00EF20FB
:0602D0005921592108002C
:00000001FF
